:020000040800F2
:10000000C8040020D9000008D11400081314000807
:1000100000000000000000000000000000000000E0
:1000200000000000000000000000000005180008AB
:100030000000000000000000191500080718000863
:10004000EB000008EB000008EB000008EB000008E4
:10005000EB000008EB000008EB000008EB000008D4
:1000600000000000EB000008EB000008EB000008B7
:10007000EB000008EB00000800000000EB000008A7
:1000800000000000EB00000800000000000000007D
:10009000EB00000800000000EB000008EB00000887
:1000A000EB000008EB000008EB000008EB00000884
:1000B000EB000008EB00000800000000000000005A
:1000C0000448854600F04AFB00480047D92500084F
:1000D000C046C046C8040020044880470448004782
:1000E000FEE7FEE7FEE7FEE7FEE7FEE77918000819
:1000F000C100000830B50B46014600202022012433
:1001000009E00D46D5409D4205D31D469540491B4B
:100110002546954040191546521E002DF1DC30BD94
:10012000F0B51FB40646002082B005464024019178
:1001300000901BE0019922460F46304600F0F3F88C
:10014000049A059B801A994110D3104619462246FD
:1001500000F0D9F8361A8F4101972246012000217C
:10016000009F00F0D0F838184D4100902046641EE2
:100170000028DFDC019B00982946324607B0F0BD1D
:10018000D2B201E00270401C491EFBD2704700222F
:10019000F6E710B513460A4604461946FFF7F0FF86
:1001A000204610BDF8B502464A40D40F42004B002D
:1001B00052085B089A4202D20246084611464A009B
:1001C00023D0C30D4A00DDB2120EAD1A202D35DA50
:1001D00049020126490AF6058A19002C00D052422C
:1001E00020214F1B1146B9402A411018C20D9A42D6
:1001F00021D0002C17D0012D08DCDA05801AD20F8F
:100200008019D207DBB200F0A7F8F8BDDA05801A32
:10021000012340001B06C01880185A428018CA0FDC
:100220001043490007E04908C2071143DA05801A64
:1002300080194008801800F087F8F8BD610001229D
:10024000511A001BF7E70122D2075140AAE7012209
:10025000D2075040A6E7024670B54A40D30FDB07ED
:1002600040002DD04A002AD0010E140E00021202C6
:100270000919400A520A8418E50104465443000A49
:10028000120A2E045043A4194219200CC543AA187F
:10029000120C0125AD03521C521912047F3924049B
:1002A00000D0521C104301D44000491EC2B20C06BB
:1002B000C0092018401C4008802A02D003E000201A
:1002C00070BD40084000002900DA0020184370BDCE
:1002D00010B500229623114600F03EF810BDC20F63
:1002E000D207400040080BD0C10D0723DB01C9181D
:1002F00040020905400A1143C208400711437047F4
:1003000000200146704710B5202A04DB0146203A40
:100310009140002010BD914020239C1A0346E340E9
:100320001943904010BD10B5202A04DB0846203A3E
:10033000D040002110BD0B46D340D0402024A21A4B
:1003400091400843194610BD002904DA401C4900B9
:1003500001D140084000704770B40024050C05D15D
:100360001024000402D1002921D01124050E01D14E
:1003700000020834050F01D10001241D850F01D1B1
:100380008000A41C002801DB4000641C002908D068
:1003900020252E1B0D46F540A14000D00121294308
:1003A000084301061B1B000ADB1D02D5002070BCA0
:1003B0007047DB05181880180029F8DA401C49003E
:1003C000F5D170BC4008400070470000F0B507460A
:1003D0000846584087B0C00F049048000E465900A8
:1003E00040084908BC1A884105D2384631461E46A5
:1003F00017460B4602465800400810434DD0300DBA
:10040000039040055900400D490D0590401A029097
:10041000402873DA18030121000B090508430190F5
:1004200004980092002806D01146019A4942002003
:10043000904100910190029840210A1A0199009878
:10044000FFF761FF05460C466B4607CB00F098F9B5
:10045000C0197141039A0E0D0023D71756401A4652
:100460007A40164344D0049A002A2DD0029A012AD9
:10047000039A15DC1205C01A914101263605001CAD
:100480007141D20F059ED2070093019202962A462F
:10049000234600F095F907B0F0BD38463146FAE73B
:1004A0001605234A0F46B218C01AB74101210905A3
:1004B000001C4F4100187F41114618187941E20F86
:1004C00010436D19644113E0E2076D081543640899
:1004D000C2071443039A01261205C01A914136053A
:1004E000001C7141CE07400830434908C0185141F3
:1004F0002A46234600F057F9CDE7FFE7049801228A
:100500004000C117121A00238B4104983146C417CA
:10051000381AA141EEE730B40124E407634030BC4F
:1005200054E730B40124E407614030BC4EE70000DA
:100530000000E0FFF0B51FB488B00B9909980024C3
:1005400048400999C00F490049080991C0070B9913
:100550000090490049080B9109990898A64608435C
:100560001CD00B990A98084318D009980124400020
:10057000420D4800410D099824050003000B20435B
:1005800009900B980003000B20430B9050181C4956
:100590004018002201901446104605E00020014654
:1005A0000DB0F0BD032801DA034600E003239C46AA
:1005B000C11A0AAE0AE05F0008ADED5B4F00F75BC1
:1005C0007D430027AA187C41491C5B1E6145F2DD72
:1005D000410004AB5A522104120C0A43240C401C63
:1005E0000828DFDB01980290009970460191009085
:1005F000059B049A0799069800F0E2F8D0E70000FE
:100600000DFCFFFFF0B50C465C4085B0E40FE4073D
:1006100003944C0000266408590094464908024699
:100620000296224321D062460A431ED06200570D33
:100630004A000E032303550D012402462C492405CC
:10064000781B1B0B360B4018234326436146009052
:100650001C46501AB44103D30098401C009002E09D
:10066000921800985B41002803DA0020014605B08B
:10067000F0BD0020012109050746864611E06446C9
:100680001D46141BB54106D36546521BB341744643
:1006900007430C43A646CD07400849082843921853
:1006A0005B4105460D43EAD11046184313D060461E
:1006B000194650407140084306D06046101AB341B5
:1006C00006D20122002306E000220123DB0702E01C
:1006D0000122D2435310009874460105381C614131
:1006E000029C039D0019694100F05DF8BFE700001E
:1006F000FD0300004A0009030123090B1B051943F0
:100700000A4B10B5520D9A4202DA0020014610BD84
:10071000064B34339A4203DC9A1AFFF704FE10BDED
:10072000034BD218FFF7EFFD10BD0000FF030000E0
:10073000CDFBFFFF10B5002904DB0124E407404294
:100740008C412146002B04DB1C460123DB0752426F
:10075000A341994200D1904210BD0000064C0125F2
:10076000064E05E0E36807CC2B430C3C9847103459
:10077000B442F7D3FFF7A8FCA0260008C026000863
:1007800010B5202A06DBCB170846203A1041C117C6
:100790000B4306E00B461341D0402024A21A91409F
:1007A0000843194610BD10B5002B08DA0024401C80
:1007B000614192185B411A4301D14008400010BDCD
:1007C000F0B51FB482B005460C0003D0084601F016
:1007D00069FA02E001F066FA2030024600902146F4
:1007E0002846FFF790FD049B059A04460F461843E0
:1007F0001143084314D0184610431BD000984021E1
:100800000A1A18460599FFF78EFD05460E46009A0E
:1008100005990498FFF777FD084305D0012004E00F
:100820002046394607B0F0BD0020C11705430E43EE
:100830002C43374300990E986305401A7905E40A62
:1008400000220C43FD0A0A3002D500200146E9E7E8
:100850000105101969410C9C0D9D00196941FFF7B4
:10086000A2FFDFE7704770B5044600F0D3F80546F5
:10087000601C00D0641C00F0CDF8401BA042FAD3ED
:1008800070BD0000F8B500230124A2E027469F4078
:100890003A4070D04D68022D01D0122D14D1DD08E0
:1008A000AD002D1800952D6A5E07AC46F50E0F269B
:1008B000AE46AE406546B543AC460E697546AE40A1
:1008C00065462E43009D2E624D68012D05D0022DF8
:1008D00003D0112D01D0122D16D185680326AC4608
:1008E0005D00AE46AE406546B543AC46CE68754643
:1008F000AE4065462E43866046680D79BE43ED06E0
:10090000ED0F9D403543456006685F000325BD40FF
:10091000AE46AE430D79B446AE07B60FBE4065464F
:100920002E430660C6687546AE438D68BD403543AC
:10093000C5604D68ED004BD5294D6E6B26436E6347
:100940009E08284DB6007519AC46AD689E07360F57
:100950000F27B740BD4305273F07B84201D1002705
:1009600015E0214FB84201D1012710E01F4FB842D6
:1009700002D102270BE02BE01D4FB84201D1032723
:1009800005E01C4FB84201D1052700E00627B7401B
:100990002F436546AF60184D2E684F689643FF039E
:1009A00000D516432E606E684F689643BF0300D58E
:1009B00016436E60AE684F689643FF0200D516433B
:1009C000AE60EE684F689643BF0200D51643EE60F6
:1009D0005B1C0A681546DD4000D057E7F8BD0000F3
:1009E00000100240000001400004005000080050C8
:1009F000000C0050001C0050000401400069084039
:100A000000D001207047002A01D0816170478162C7
:100A1000704700000148006870470000380000205F
:100A200002480168491C016070470000380000203E
:100A300010B5084800240168402211430160204697
:100A400000F00AF8002801D0012401E000F01CF8B1
:100A5000204610BD0020024070B5054609487D21A2
:100A60000024C9000068FFF745FB00F0EFFB0028F9
:100A700001D0012404E000222946501E00F010F8A5
:100A8000204670BD3C0000200448416B0122114308
:100A90004163816B0204114381637047001002407F
:100AA00010B500F017FD10BDF8B504460078544DA0
:100AB000800672D5524E0027403EB06BC00004D471
:100AC000B06BA9050843B06301274E480168C9050A
:100AD00011D40168821511430160FFF79BFF00905C
:100AE00005E0FFF797FF0099401A642837D845487A
:100AF0000068C005F5D532680321090560680A4021
:100B00000140914208D08103890F032904D1316843
:100B1000890301D50120F8BD2A69032109040A408F
:100B200022D0084090421FD0207880061CD528692A
:100B30002A6988430121C9040A432A612A698A4330
:100B40002A612861C0050FD5FFF764FF009008E017
:100B5000FFF760FF0099411A2B48814201D9032019
:100B6000F8BD28698005F3D561688803800F0328E4
:100B700005D132680005824301400A43326028698A
:100B8000032261681204114008432861002F04D039
:100B9000B16B012000078143B1632078C00705D005
:100BA000E868A168800880000843E8602078800732
:100BB00005D5E8680C218843E1680843E86020789F
:100BC000400706D5E8680321890288432169084364
:100BD000E8602078000706D5E86803210903884308
:100BE00061690843E8602078000606D5E8680321BB
:100BF00089048843A1690843E8600020F8BD00002B
:100C0000401002400070004088130000F8B50E4606
:100C100005007DD053480068C007C00FB0420AD21B
:100C20005048016849084900314301600068C00725
:100C3000C00FB04271D128784B4C800705D5E068D1
:100C4000F0218843A9680843E0602878C00752D0A3
:100C50006868022817D0032818D02168012818D006
:100C60008905002959DAE168890889000143E160B2
:100C7000FFF7D0FE69680746022912D003291CD06D
:100C8000012926D033E021688903EAE72168890138
:100C9000E7E74907E5E7FFF7BDFEC11B334881429F
:100CA00023D8E0680007800F0228F4D123E0FFF783
:100CB000B1FEC11B2D48814217D8E0680007800FA4
:100CC0000328F4D117E0FFF7A5FEC11B2748814296
:100CD0000BD8E0680007800F0128F4D10BE0FFF784
:100CE00099FEC11B2148814201D90320F8BDE0686B
:100CF0000007800FF3D11B480168C907C90FB14233
:100D00000DD901684908490031430160006800E0DD
:100D100003E0C007C00FB04201D00120F8BD287821
:100D2000400706D5E068072109028843E9680843BF
:100D3000E0602878000707D5E0680721C9028843EA
:100D40002969C9000843E06000F036F8E168084A04
:100D50000906090F515CC840064908600020FFF7EA
:100D60007BFEF8BD00200240001002408813000006
:100D70007C2600083C000020044805490068C9683A
:100D8000044A4905490F515CC84070473C000020A7
:100D90000010024095260008044805490068C9680B
:100DA000044A8904490F515CC84070473C00002048
:100DB000001002409526000810B5184AD1680C2092
:100DC000084004280BD0082810D00C2810D05068F8
:100DD0000004410F0120C003491C884010BD106869
:100DE000C00601D50E4810BD0E4810BD0E4810BDFE
:100DF00088020E4B000F185C0902D368890F491C4A
:100E0000DB0301D5084A05E01268D20601D5044A81
:100E100000E0044A5043FFF76DF910BD0010024096
:100E200000093D000024F40000127A008C2600081E
:100E3000FEB505007ED0FE4CE7680C20E668074052
:100E40000120000406402878C00747D0082F05D0AD
:100E50000C2F0AD101200004864206D120688003AD
:100E60003CD568680028E5D038E0012069680004B6
:100E7000814203D121680143216011E00523012251
:100E80001B0492049942216802D111432160F1E7C9
:100E900081432160216801400091206890432060D7
:100EA000686800280DD0FFF7B5FD009005E0FFF75A
:100EB000B1FD0099401A64287AD820688003F6D5DD
:100EC0000CE0FFF7A7FD009005E0FFF7A3FD0099F8
:100ED000401A6428F0D820688003F6D42878800768
:100EE00055D50923E868042F0DD00C2F01D1002E11
:100EF00009D000283BD02168994301432160FFF7C6
:100F000089FD064627E02168490701D5002891D0D0
:100F100061681F22120291432A6912021143616023
:100F20002168994301432160FFF746FFE168090604
:100F30000A0F00E079E1BF49895CC840BE490860FA
:100F40000020FFF789FD002872D120E0FFF762FD45
:100F5000801B0228B0D820684007F7D560681F21A1
:100F60000902884329690902084360600FE020688C
:100F7000400840002060FFF74DFD064604E0FFF703
:100F800049FD801B022897D820684007F7D42878AD
:100F9000C0065FD5002F0CD0A869002849D0206872
:100FA000FF21013108432060FFF734FD06462DE0A4
:100FB000C0E02068800502D5A8690028A7D0606835
:100FC000072149038843296A084360606068297FD4
:100FD0000002000A090608436060286A410B0120EC
:100FE000C003491C8840E16809060A0F9149895CE1
:100FF000C840914908600020FFF72EFD002817D156
:1010000028E0FFF707FD801B0228A3D82068800591
:10101000F7D56068072149038843296A084360605F
:101020006068297F0002000A09060843606011E039
:10103000E1E02168FF20013081432160FFF7EAFCF5
:10104000064604E0FFF7E6FC801B022872D8206801
:101050008005F7D42878794E000724D568690028E0
:10106000306910D0012108433061FFF7D3FC0090B4
:1010700005E0FFF7CFFC0099401A02285AD83069E2
:101080008007F6D50FE0400840003061FFF7C2FC52
:10109000009005E0FFF7BEFC0099401A022849D8ED
:1010A00030698007F6D42878400765D50020029083
:1010B000A06BC00006D4A06B012109070843A06300
:1010C000012002905E480168C90511D401688215AB
:1010D00011430160FFF79EFC009005E0FFF79AFCCA
:1010E0000099401A642825D855480068C005F5D5F0
:1010F000FF20AA680130824203D131690143316186
:1011000011E001218902002A07D005231B029A421F
:1011100003D132690A433261EFE7326982433261B7
:10112000306988433061A86800280FD0FFF772FC4F
:10113000009007E05EE0FFF76DFC0099411A41481E
:10114000814257D830698005F5D50DE0FFF762FC84
:10115000009006E0FFF75EFC0099411A3948814291
:1011600048D830698005F5D40298002804D0A06BD7
:10117000012109078843A063686A002864D00C2F06
:101180003ED0012636060228206805D0B0432060F4
:10119000FFF740FC05462FE0B0432060FFF73AFC24
:1011A000074604E0FFF736FCC01B022822D820685F
:1011B0008001F7D4E96AA86AE2680843296BFD2335
:1011C0001B049A4311430843E060206830432060C9
:1011D000FFF720FC054604E0FFF71CFC401B02283B
:1011E00008D820688001F7D52EE0FFF713FC401BDC
:1011F000022801D90320FEBD20688001F5D423E038
:101200000128F8D0E06801210904AA6A014091424E
:101210000BD10F218904EA6A0140914205D10321D3
:1012200089050840296B88420ED00120FEBD0000D0
:10123000001002407C2600083C00002040100240C4
:1012400000700040881300000020EFE7094910B546
:10125000401E884201D9012010BD074C6061032166
:10126000081F00F037F90020A0610720206100204E
:1012700010BD0000FFFFFF0000E000E010B504001B
:1012800003D0606F002802D007E0012010BD0021CC
:1012900070200155204600F027F824206067206860
:1012A0000168490849000160204600F0A5FB0128BB
:1012B000ECD0606A002802D0204600F007FB2068CE
:1012C00041680922D20291434160206881682A2244
:1012D000914381602068016801221143016020462A
:1012E00000F05AFB10BD000010B586B00446142172
:1012F0006846FEF74CFF1149206888421CD110480F
:10130000416B0122920311434163C16A01221143DF
:10131000C162C06A694610400590032040020090F7
:1013200002200190002002900320039004200490EA
:1013300005200007FFF7A6FA06B010BD00380140EF
:1013400000100240FFB50446406F83B017460D46BB
:1013500020285CD1002D0AD0002F08D0A168C00140
:10136000814207D12069002804D1E80702D001207A
:1013700007B0F0BD204660300290007C012846D0C6
:101380000298012101740020E06721206067FFF7C7
:1013900041FB264640360190378277820120A168C2
:1013A0000003814202D12069002802D02F46002587
:1013B00011E000270FE000228021204600F030FCE1
:1013C000002815D1002F15D02168387888627F1C3D
:1013D000708A401E7082708A019B002806980090D7
:1013E000E9D100224021204600F01AFC002808D054
:1013F0000320BDE728882168C005C00D8862AD1CA8
:10140000E6E720206067029900200874B0E7022018
:10141000AEE7FEE730B587B014216846FEF7B7FEA9
:101420000D48C16A01242143C162C06A05252040DC
:101430002D070590002230212846FFF7E4FA00210D
:101440003020029103910090019469462846FFF7ED
:1014500019FA07B030BD00000010024000B587B097
:1014600014216846FEF793FE0A48C26A08210A431F
:10147000C262C06A084005901020009000200190D0
:1014800002200290052069460007FFF7FBF907B02C
:1014900000BD00000010024010B50C480A49016070
:1014A000E1214902416000218160C16001618161E7
:1014B000C1610C22016242614162FFF7DFFE002838
:1014C00001D0FFF7CFF910BD0038014044000020E3
:1014D000704700008307FF22DB0E9A408907090E40
:1014E000994000280BDA0007000F083883080848E5
:1014F0009B001818C36993430B43C361704783086B
:1015000004489B001B1818689043084318607047F4
:1015100000ED00E000E400E070470000FEB5274C5D
:101520002089FEF7D5FEE169FEF795FEA169FEF779
:1015300039FE074660636089FEF7CAFE00900546E3
:101540006169FEF788FE2946FEF785FE054600988C
:101550002169FEF780FEE168FEF724FE2946FEF7CA
:1015600021FEE06206460098616AFEF774FE216A79
:10157000FEF718FE054612493846FEF764FE294676
:10158000FEF769FE3146FEF70DFE0E4920638842E4
:1015900002DC0D49884200DA2163206BFEF79FFED2
:1015A00004460D463846FEF79AFE02460B4607A053
:1015B0000195009400F066FBFEBD000000000020D5
:1015C0000000C8410000C842CDCCCC3D25332E31AF
:1015D0006625332E3166000070B5214C00206080F6
:1015E000FFF73CFF8020052520802D070A20FFF70C
:1015F0003AF9012220212846FFF705FA0A20FFF7D1
:1016000032F910212846FFF7F9F9002803D0608845
:10161000218808436080002220212846FFF7F3F943
:10162000208840082080E1D1FFF7F4FE002210213D
:101630002846FFF7E8F90A20FFF715F901222021D3
:101640002846FFF7E0F90A20FFF70DF900222021D4
:101650002846FFF7D8F90A20FFF705F970BD00000A
:101660000000002010B5FFF7D5FE05242407012255
:1016700010212046FFF7C7F9002220212046FFF75E
:10168000C2F90A20FFF7EFF8012220212046FFF7D8
:10169000BAF90A20FFF7E7F8002210212046FFF7E9
:1016A000B2F90A20FFF7DFF8002220212046FFF7D9
:1016B000AAF90A20FFF7D7F8012220212046FFF7D8
:1016C000A2F90A20FFF7CFF8012210212046FFF7E8
:1016D0009AF90A20FFF7C7F8002220212046FFF7D9
:1016E00092F90A20FFF7BFF810BD000070B5FFF7B0
:1016F00091FE80201F4C052520802D072078800733
:1017000001D0012200E0002210212846FFF77BF9DA
:101710000A20FFF7A8F8012220212846FFF773F9D5
:101720000A20FFF7A0F8002220212846FFF76BF9D6
:101730000A20FFF798F8208840082080DED1FFF7C4
:101740008DFE0A20FFF78FF8012220212846FFF79F
:101750005AF90A20FFF787F810212846FFF74EF9BB
:10176000A062002220212846FFF74DF90A20FFF74A
:101770007AF870BD0000002070B5FFF74BFE8020A6
:101780001F4C05262080350780B2304201D001224F
:1017900000E0002210212846FFF735F90A20FFF764
:1017A00062F8012220212846FFF72DF90A20FFF7D1
:1017B0005AF8002220212846FFF725F90A20FFF7D2
:1017C00052F8208840082080DED1FFF747FE0A202B
:1017D000FFF749F8012220212846FFF714F90A20D3
:1017E000FFF741F810212846FFF708F9A062002210
:1017F00020212846FFF707F90A20FFF734F870BDCB
:1018000000000020704710B5FFF70AF910BD000076
:1018100030B599B034216846FEF7B9FC14210DA803
:10182000FEF7B5FC1C2112A8FEF7B1FC11480168B7
:101830000322D2029143C214891801600220009051
:101840000024102009940125049003956846FFF7B1
:10185000EFFA0F200D900F94109400210E95119423
:101860000DA8FFF7D3F912A812951494FFF71CF9ED
:1018700019B030BD00700040104801688215114356
:101880000160C1680E4A1140C16001680D4A1140F3
:101890000160816849084900816001680122920461
:1018A00091430160C168FD2212049143C16000218F
:1018B00001610549C00388607047000000100240C4
:1018C0000C40FF88F6FFF6FE00ED00E010B5818CBD
:1018D000C90707D001684A6801235B049A43836AF9
:1018E0001A434A60818C890707D501684A68012339
:1018F0001B049A43C36A1A434A60818C490707D57F
:1019000001684A6801239B049A43036B1A434A60A7
:10191000818C090707D501684A680123DB039A43D4
:10192000436B1A434A60818CC90607D502689168E7
:1019300001231B039943836B19439160818C8906B2
:1019400007D501688A6801235B039A43C36B1A4376
:101950008A60818C490612D503685A6801210905FD
:10196000046C8A4322435A60026C8A4207D102689F
:10197000516803235B059943436C19435160818C83
:10198000090607D501684A680123DB04806C9A4385
:1019900002434A6010BD0000F8B500260446C66741
:1019A000FFF738F8054620680068124F000709D590
:1019B00001212B46002249052046009700F030F90E
:1019C00000280DD12068006840070BD501212B4667
:1019D000002289052046009700F022F9002801D056
:1019E0000320F8BD20206067A067603426740020C3
:1019F000F8BD0000FFFFFF01F8B504462669A268A4
:101A0000E76932436669102000253E43236832436C
:101A100078491E68784F3E4016431E6023685A6816
:101A200003263603B243E66832435A602368A2694C
:101A30008B4201D0266A32439E680B273F02BE4389
:101A400016439E606D4E23686D4AB3420CD1D26836
:101A50009207920F06D0012A38D0022A34D0032AE6
:101A600020D11EE001201DE0664EB3420AD1D268AB
:101A70000C26324026D0042A28D0082A24D00C2A4A
:101A800010D10EE08B420DD1D6680322920216408F
:101A900018D001229202B61A18D0B61A14D0964263
:101AA00000D10820564A0126403A574FF6038B4290
:101AB00036D100280CD002280DD0042812D00828D6
:101AC0001FD11CE00020EDE70220EBE70420E9E74E
:101AD000FFF752F908E01068C00601D5384605E066
:101AE0004A4803E0FFF768F9002873D062685100A4
:101AF0005118814205D81103814202D303E03046D8
:101B0000F4E7012566E0010E0602500800233018B4
:101B10005941FEF705FB03210902411A3C4A55E0F1
:101B2000E169B14232D1030000F0D3F809070A0D90
:101B300006250606062B0600E3E7FFF71DF91CE065
:101B4000FFF72AF919E010686168C00602D5480855
:101B5000304A01E0304A48088018FEF7CBFA80B2DC
:101B600001462E4A10399142CBD8511C0140000742
:101B7000400F08432CE0FFF71FF9616840004A0856
:101B8000EAE76168012248081204E5E7030000F073
:101B9000A0F809070A0D06260606062C0600B0E77F
:101BA000FFF7EAF81DE0FFF7F7F81AE01068616840
:101BB000C00602D54808C01902E014484A081018A7
:101BC000FEF798FA80B20146144A1039914298D82B
:101BD0002168C8600020206660662846F8BDFFF7CF
:101BE000EBF861684A088018EAE7616848088019DC
:101BF000E6E7000000480040F369FFEF00380140CD
:101C0000401002400044004000093D000024F40060
:101C1000FFFC0F0000127A000048E801EFFF00000F
:101C2000FFB581B017460E4604460A9D09E0681CC0
:101C300007D0FEF7EFFE0499401AA8420CD8002DF9
:101C40000AD02068C1693046884318D00020B842C5
:101C5000EDD0002005B0F0BD20680168FF22A13260
:101C60009143016020688168490849008160202013
:101C70006067A0670020603420740320EAE7012039
:101C8000E5E700000FB410B503A9044B044A02981D
:101C900000F0F6F810BC08BC04B01847BD250008D9
:101CA000400000202021020C01D010211046020A21
:101CB00001D010460839020901D01046091F8208D8
:101CC00001D01046891E420801D0881E7047081AAC
:101CD000704730B47446641E2578641CAB4200D251
:101CE0001D46635D5B00E31830BC184702E008C87E
:101CF000121F08C1002AFAD170477047002001E086
:101D000001C1121F002AFBD170470000F0B51FB4BB
:101D100086B00998089A030D0021024314D0514857
:101D2000514A1818504305141198012810981AD0D8
:101D3000281A401C00264D4F4D49009601910490F1
:101D4000002812DA444211E01198012449A3012825
:101D500001D11098C1430698119A84600360C26053
:101D600041600BB0F0BD4042E4E70446210500208D
:101D70003F4A001C51410391029012E0E00707D056
:101D800032463B4601990098FEF7D4FB0191009042
:101D900032463B4610461946FEF7CCFB06460F4638
:101DA0006410002CEAD10498039B0028029A099938
:101DB000089806DAFEF7BEFB019B009AFEF7BAFB15
:101DC00005E0FEF71FFC019B009AFEF71BFC044692
:101DD0000E460022284BFEF7ADFC03D80020C0437E
:101DE000014607E00022254B20463146FEF7EEFA79
:101DF000FEF780FC102409E0002C0ADB0A220023F5
:101E0000FEF78EF9079B30321A55641E02460A43CC
:101E1000F2D11122641C079B121B1C19119B012B70
:101E200003D0012308430ED10AE0084304D0112057
:101E300010900020119077E71098151A6D1E0BE096
:101E40001098824202DD00236D1C03E0824201DA19
:101E500000236D1E002BEED0069811998260C160A0
:101E600030C07EE701FCFFFF104D00000000144071
:101E70000000F03F300000000000F0430000E03FB1
:101E8000FFB597B0064600251BE2252876D1002431
:101E90002746F749049400E00443761C3278012079
:101EA000203A90400842F7D130782A280ED00222FA
:101EB000307801463039092916D804990A23594344
:101EC000303940181443761C0490F1E7189802C882
:101ED00004911890002904DA012040030443484289
:101EE000049002200443761C30782E2814D104205C
:101EF00004437078761C2A2809D11898761C80C86B
:101F0000189009E00A214F43303FC719761C3078FA
:101F1000014630390929F5D930786C2810D006DC13
:101F20004C281AD068280ED06A2817D104E07428EB
:101F300013D07A2812D110E00120400504430CE0B0
:101F40000121090501E0032109050C437178814253
:101F500003D1012000052418761C761C30786628F1
:101F60000BD013DC58287DD009DC00287BD0452815
:101F7000F6D04628F4D047281AD1A9E118E0632802
:101F800035D0642870D0652812D1A1E170286CD0BA
:101F900008DC6728F1D069287DD06E280DD06F2825
:101FA00006D1BCE073282ED0752873D0782859D07C
:101FB0001A9A199990476D1C82E16002400F02281D
:101FC00009D003280DD00428189801680DD00D60A1
:101FD000001D189074E11898EA1701680D604A60B6
:101FE000F6E7189801680D80F2E70D70F0E7189891
:101FF0006A4601781172001D18900020507202A8E4
:102000000090012005E0189802C818900020009167
:10201000C04361070ED5002101E00199491C0191DF
:10202000B94213DA8142F8DB019A0099895C0029F0
:10203000F3D10BE0002101E00199491C019181429B
:10204000FADB019A0099895C0029F5D1019904987D
:102050001A9B471A21463846199A00F099FA4019F6
:10206000019903E051E030E115E050E0451807E048
:10207000009800990078491C00911A9A1999904784
:102080000198401E0190401CF2D1214638461A9B0F
:10209000199A12E137E00A200021009001916002B4
:1020A000410F022907D0189A01CA1892C217944604
:1020B000032908D00AE01898C01DC108C90005C945
:1020C0001891944607E000B2C2179446042902D141
:1020D00040B2C1178C4600226146944506DA0A4692
:1020E0000021404291418C462D2102E0210504D57A
:1020F0002B216A461173012103E0E10701D0202161
:10210000F7E7029156E00A200AE0102008E01020CC
:1021100000900021042004430191082703E00820D7
:102120000021019100906002410F022907D0189A06
:1021300001CA189200229446032908D008E0189892
:10214000C01DC108C90005C91891944603E080B2BA
:10215000042900D1C0B20021029121072AD531788B
:102160000D91702906D0009A1021019B4A401A4314
:1021700005D00EE040216A461173012108E0614656
:10218000014306D030216A4611730D995173022123
:102190000291009A0821019B4A401A430AD16146E4
:1021A000014301D1610705D530216A461173012130
:1021B0007F1E02913178582904D02EA10E910DA9CD
:1021C0000D910DE030A1F9E76146019B009AFDF702
:1021D000A7FF0E9B8C469B5C0D9A521E0D921370AE
:1021E00061460143F0D10D9805A9081A20300190ED
:1021F000600703D501200004844300E00127019813
:10220000874201DD381A00E0002001990090411852
:10221000029809180498401A0490E00306D4214655
:102220001A9B199A049800F0B3F94519002706E0A3
:1022300003A81A9AC05D199990476D1C7F1C0298DB
:102240008742F5DBE0030CD521461A9B199A0498C6
:1022500000F09EF9451904E01A9A30201999904728
:102260006D1C0099481E00900029F5DC1FE000005D
:10227000092801003031323334353637383961625C
:102280006364656600000000303132333435363720
:102290003839414243444546000000000D980D99ED
:1022A0000078491C0D911A9A199990476D1C019953
:1022B000481E01900029F1DC4DE100F059F9451963
:1022C000761C3078002800D0DFE528461BB0F0BD32
:1022D000600700D406271898C01DC108C9004868C7
:1022E0000A680831C30FDB071891190001D09CA1BF
:1022F00008E0210501D59BA104E0E10701D09AA1E6
:1023000000E09AA14300109130785B0865280CD05A
:1023100006DC452809D046281DD0472841D141E098
:10232000662818D067283CD13CE00021112F01DB42
:10233000112000E0781C0191009008A911A8FFF776
:10234000E5FC139905910021119A15927F1C1298B2
:102350000197009150E00120C007039001200190F7
:1023600008A9009711A8FFF7D1FC139A14990592B8
:102370000022119B009212981593059A0192002950
:1023800001D0104602E0791C40180190381A01D59E
:10239000019804E04042401E0090781C0190C01B50
:1023A000029043E0012F00DA01270021112F01DD07
:1023B000112000E038460191009008A911A8FFF70C
:1023C000A5FC13990591119A00211298159200917C
:1023D000019721070CD40599B94201DB019900E06E
:1023E0000191012904DD159A491E515C302906D05E
:1023F000B84201DA011D05DA0121029115E00199C7
:10240000491EEDE7002805DC00994118009101996B
:10241000091A03E0019A411C914200DD01910099E3
:10242000401A401C02900120C0070390200706D4E8
:1024300002990198814202DB0020C04302900020F3
:102440006946C87707AF012103980337C907884257
:1024500024D0022011902B201290039800280CDA2F
:10246000404203902D20129007E00A210398FDF7C7
:1024700041FE30317F1E039039701199481E119032
:102480000029F2DC03980028EFD1791E1298087019
:102490003078202108404530BF1E387006A8C01B88
:1024A000C01D039010980078002800D001200199E9
:1024B00041180298C0170918039809180498401A7F
:1024C000401E0490E00306D421461A9B199A0498F2
:1024D00000F05EF8451910980078002803D01A9A89
:1024E000199990476D1CE00324D521461A9B199A2F
:1024F000049800F04DF845191CE00098002807DB0F
:1025000000990598884203DD1598405C199901E00F
:10251000199930201A9A904700986D1C401C009021
:102520000298401E0290002804D11A9A2E20199970
:1025300090476D1C0199481E01900029DDDC05E0E3
:1025400038781A9A7F1C199990476D1C0399481E78
:1025500003900029F4DC21461A9B199A0498ACE6F2
:102560002D0000002B0000002000000000000000F3
:10257000F8B5044600251E461746880404D405E035
:1025800039462020B0476D1C641EF9D52846F8BD99
:10259000FFB50446002581B01E46C80301D530278B
:1025A00000E02027880404D505E038460399B047A9
:1025B0006D1C641EF9D5284605B0F0BD13B5044B5B
:1025C000012269460348FEF7BDFE00981CBD0000CD
:1025D000FFFF000044000020FEF72AFAFFF718F979
:1025E000FEF718FFFEF758FF00250526214C224F65
:1025F000360725816581A580E580FFF733F8FFF771
:1026000075F8FEF72BFFFA20FEF72DF91021304662
:10261000FEF7F4F900280BD1FEF7DEFF6088A080FA
:10262000FEF7DAFF6188E18020790002084320810B
:10263000FFF718F8FFF7A0F8FEF710FFFA20FEF7F3
:1026400012F910213046FEF7D9F900280BD1FEF718
:10265000C3FF6088A080FEF7BFFF6188E18020791A
:10266000000208436081FEF759FF3846FEF7FBF889
:10267000BFE7000000000020C409000000000000C7
:10268000000000000102030406070809030406080D
:102690000C101820300000000001020304000000AC
:1026A000C02600080000002044000000EC1C0008C8
:1026B000042700084400002084040000FC1C0008DB
:1026C000000000000000000000000000C5FE02C085
:1026D000BD52163DF624D6B566661EC20AD7233C07
:1026E0000AD7233CACC5A73800000000000000005A
:1026F00000000000000000000000000000002000BA
:0427000000000000D5
:04000005080000C12E
:00000001FF
